:100074009307000063880700371500001305C515B2
:100084006F10401367800000130101FF23248100D7
:1000940083C7C1C32326110063920702930700009C
:1000A400638A0700372500001305C539970000004F
:1000B400E700000093071000238EF1C28320C100E3
:1000C40003248100130101016780000093070000ED
:1000D400638C070037250000938501C41305C539D7
:1000E400170300006700000067800000130101FF90
:1000F400232681001304010183A7C1C293878700CB
:1001040003A7070023AAE1C283A741C393F71700FB
:1001140093B7170093F7F70F138507000324C10063
:100124001301010167800000130101FF23268100F0
:100134001304010183A7C1C29387870003A70700A3
:1001440023AAE1C203A741C3B7070100B377F700AD
:1001540093B7170093F7F70F138507000324C10023
:100164001301010167800000130101FE232E8100A9
:10017400130401022326A4FE83A7C1C29387870028
:1001840003A7070023AAE1C283A741C393F717007B
:10019400639E070083A7C1C2938747000327C4FE59
:1001A40023A0E700930700006F0080009307F0FF8F
:1001B400138507000324C1011301010267800000B5
:1001C400130101FF232681001304010183A7C1C287
:1001D4009387870003A7070023AAE1C203A741C3AB
:1001E400B7070100B377F7006398070083A7C1C27C
:1001F40083A707006F0080009307F0FF13850700B3
:100204000324C1001301010167800000130101FEF2
:10021400232E1100232C8100130401022326A4FEA3
:100224006F000003130000008327C4FE83C7070088
:1002340013850700EFF05FF3130705009307F0FF42
:10024400E304F7FE8327C4FE938717002326F4FEF6
:100254008327C4FE83C70700E39607FC93070000C7
:10026400138507008320C1010324810113010102C6
:1002740067800000130101FD23261102232481025B
:1002840013040103232EA4FC232CB4FC232604FE14
:10029400032784FD9307100063C6E700930700005B
:1002A4006F008009EFF0DFF12324A4FE032784FE0E
:1002B4009307F0FFE308F7FE8327C4FE13871700B4
:1002C4002326E4FE138707008327C4FDB387E700D2
:1002D400032784FE1377F70F2380E7001300000041
:1002E400032584FEEFF05FE8130705009307F0FF92
:1002F400E308F7FE832784FD9387F7FF0327C4FEF3
:100304006350F702032784FE9307A000630CF700F1
:10031400032784FE9307D0006306F7006FF09FF86D
:10032400130000008327C4FE0327C4FDB307F700AE
:10033400238007008327C4FE138507008320C1029E
:10034400032481021301010367800000130101FCEF
:10035400232E8102130401042326A4FC2324B4FCC9
:10036400232404FE232204FE832784FC63DA07008B
:10037400832784FCB307F0402324F4FC232204FEE7
:10038400832784FC63960706832784FE138717005C
:100394002324E4FE138707008327C4FCB387E70004
:1003A400130700032380E7006F008007032784FC02
:1003B4009307A000B367F70213F7F70F832784FEB0
:1003C400938617002324D4FE938607008327C4FC56
:1003D400B387D700130707031377F70F2380E700CA
:1003E400032784FC9307A000B347F7022324F4FCFB
:1003F400832784FCE34CF0FA832744FE63820702DC
:10040400832784FE138717002324E4FE1387070041
:100414008327C4FCB387E7001307D0022380E700D7
:10042400232604FE6F00C006832784FE1387F7FF8C
:100434008327C4FEB307F7402320F4FE8327C4FEBA
:100444000327C4FCB307F70083C70700A30FF4FC1A
:10045400832704FE0327C4FC3307F7008327C4FE65
:100464008326C4FCB387F600034707002380E70014
:10047400832704FE0327C4FCB307F7000347F4FDF6
:100484002380E7008327C4FE938717002326F4FE06
:10049400832784FE13D7F701B307F70093D71740D8
:1004A400138707008327C4FEE3C0E7F8832784FE8D
:1004B4000327C4FCB307F70023800700832784FEC7
:1004C400138507000324C10313010104678000009E
:1004D400130101FB23268104130401052326A4FC34
:1004E4002320B4FC2322C4FC2324D4FC9307070058
:1004F400A30FF4FA232404FE6F000009832704FCED
:1005040093F7F700232EF4FC0327C4FD9307900010
:1005140063C4E7028327C4FD13F7F70F832784FE20
:100524008326C4FCB387F600130707031377F70F7A
:100534002380E7006F0040028327C4FD13F7F70F01
:10054400832784FE8326C4FCB387F600130777054C
:100554001377F70F2380E700832744FC9397C701A1
:10056400032704FC1358470033E80701832744FC9E
:1005740093D84700232004FD232214FD832784FEFF
:10058400938717002324F4FE832704FC032744FCE9
:10059400B3E7E700E39407F66F004002832784FE85
:1005A400138717002324E4FE138707008327C4FC62
:1005B400B387E7000347F4FB2380E700032784FEA7
:1005C400832784FCE34CF7FC232604FE6F00C0065B
:1005D400832784FE1387F7FF8327C4FEB307F740FE
:1005E4002322F4FE8327C4FE0327C4FCB307F700C9
:1005F40083C70700A301F4FE832744FE0327C4FC3A
:100604003307F7008327C4FE8326C4FCB387F600B0
:10061400034707002380E700832744FE0327C4FC25
:10062400B307F700034734FE2380E7008327C4FEA3
:10063400938717002326F4FE832784FE13D7F7013C
:10064400B307F70093D71740138707008327C4FE27
:10065400E3C0E7F8832784FE0327C4FCB307F7004D
:1006640023800700832784FE138507000324C10425
:100674001301010567800000130101FD2326810297
:1006840013040103232EA4FC232CB4FC232604FE10
:10069400232404FE930710002322F4FE6F00C008F5
:1006A4008327C4FD83C707002320F4FE032704FE29
:1006B4009307F00263D2E704032704FE9307900331
:1006C40063CCE702032784FE930707009397270070
:1006D400B387E7009397170013870700832704FE67
:1006E400B307F700938707FD2324F4FE9307100054
:1006F4002326F4FE6F0080028327C4FE639E070254
:10070400032704FE9307D002631AF7009307F0FF50
:100714002322F4FE930710002326F4FE8327C4FD4E
:1007240093871700232EF4FC8327C4FD83C7070097
:10073400E39807F66F00800013000000032784FE8F
:10074400832744FEB307F7022324F4FE832784FDA2
:1007540063880700832784FD0327C4FD23A0E700E3
:10076400832784FE138507000324C10213010103B8
:1007740067800000130101FD232681021304010395
:10078400232EA4FC232CB4FC232604FE232404FEE1
:100794006F00000E8327C4FD83C707002322F4FEE5
:1007A400032744FE9307F00263DAE702032744FEBB
:1007B4009307900363C4E702930710002326F4FE13
:1007C400832784FE13974700832744FEB307F7006B
:1007D400938707FD2324F4FE6F00C008032744FE1B
:1007E4009307000663DAE702032744FE93076006D3
:1007F40063C4E702930710002326F4FE832784FED4
:1008040013974700832744FEB307F700938797FAAB
:100814002324F4FE6F000005032744FE930700041D
:1008240063DAE702032744FE9307600463C4E70224
:10083400930710002326F4FE832784FE13974700B2
:10084400832744FEB307F700938797FC2324F4FE21
:100854006F0040018327C4FE6394070293071000CE
:100864002326F4FE8327C4FD93871700232EF4FC6C
:100874008327C4FD83C70700E39E07F06F00800051
:1008840013000000832784FD63880700832784FD09
:100894000327C4FD23A0E700832784FE13850700F4
:1008A4000324C1021301010367800000130101EC5A
:1008B400232E1112232C8112232A211323283113CE
:1008C40023264113232451131304011483A781C342
:1008D40093F707FF232AF4FC232C04FC6F00401B2E
:1008E400832744FD13890700930900009307C4EC90
:1008F400130700039306800093050900138609007B
:1009040013850700EFF0DFBC9307C4EC13850700E1
:10091400EFF0DF8FB71700001385C729EFF01F8FA3
:10092400232E04FC6F00000A832744FD2326F4FCD5
:100934000327C4FD832744FD3307F70083A781C33E
:10094400637AF700B71700001385072AEFF01F8CAE
:100954006F0000058327C4FD0327C4FCB307F70019
:1009640083C70700138A0700930A0000930744EC27
:10097400130700039306200093050A0013860A0058
:1009840013850700EFF0DFB4930744EC13850700E9
:10099400EFF0DF87B71700001385472AEFF01F87B2
:1009A4000327C4FD930770006318F700B71700000E
:1009B4001385872AEFF09F858327C4FD938717004B
:1009C400232EF4FC0327C4FD9307F000E3DEE7F4D1
:1009D400B71700001385C72AEFF05F83232E04FCAA
:1009E4006F004007832744FD2328F4FC8327C4FDBC
:1009F400032704FDB307F70003C707009307F001BB
:100A040063FAE7028327C4FD032704FDB307F70055
:100A140003C707009307E00763EEE7008327C4FDDD
:100A2400032704FDB307F70083C707002300F4EC92
:100A34006F00C0009307E0022300F4EC834704EC4A
:100A440013850700EFF04FF28327C4FD9387170047
:100A5400232EF4FC0327C4FD9307F000E3D4E7F846
:100A6400B71700001385072BEFF04FFA832744FDD7
:100A740093870701232AF4FC832744FD93F7F70F98
:100A840063800702832784FD93871700232CF4FCDB
:100A9400032784FD9307F000E3D4E7E46F008000AC
:100AA40013000000B71700001385472BEFF00FF673
:100AB400032744FD23ACE1C2130000008320C113CB
:100AC400032481130329411383290113032AC11227
:100AD400832A81121301011467800000130101FFAE
:100AE400232611002324810013040101B7170000F9
:100AF4001385872BEFF08FF1B71700001385872D2F
:100B0400EFF0CFF0B71700001385C72FEFF00FF009
:100B1400B717000013854732EFF04FEFB717000007
:100B240013858735EFF08FEE130000008320C1009A
:100B3400032481001301010167800000130101E80F
:100B4400232E1116232C8116232A2117232831172B
:100B54002326411723245117130401182326A4E83C
:100B64002324B4E8B70700F0232CF4FCB70700F003
:100B740093870701232AF4FC83A7C1C29387070143
:100B84001307201B23A0E700232804FC232604FCCE
:100B9400EFF0CFD59307050063880700B71700006F
:100BA40013850737EFF08FE6EFF00FD893070500B2
:100BB400E38C07FE930744E99305F00F13850700C0
:100BC400EFF04FEB13000000B71700001385473711
:100BD400EFF0CFE3930744E913850700EFF00FE349
:100BE400B71700001385472BEFF04FE2034744E9A2
:100BF400930780066316F700EFF05FEE6F00C02ED8
:100C0400034744E9930720066316F704930744E96E
:100C1400938727009305000013850700EFF0DFA5F5
:100C24002328A4FA832704FB6352F002B7F7FA02DD
:100C340013870708832704FB3347F70283A7C1C23E
:100C44009387070123A0E7006F00002AEFF01FE954
:100C54006F008029034744E993074006631AF702AB
:100C6400930744E993872700930500001385070041
:100C7400EFF05FB0232AA4FA832744FB6356F00005
:100C8400032744FB23ACE1C2EFF05FC26F00C02531
:100C9400034744E993077007631CF70A930744E981
:100CA40093872700130784F993050700138507002A
:100CB400EFF05FAC2320A4FC832784F9130784F9A5
:100CC4009305070013850700EFF0DFAA232EA4FA8B
:100CD400832784F9130784F9930507001385070014
:100CE400EFF05FA9232CA4FA032784FB93071000D9
:100CF400631CF700832704FC0327C4FB1377F70F57
:100D04002380E7006F00401E032784FB9307200025
:100D1400631EF700832704FC0327C4FB1317070192
:100D2400135707412390E7006F00001C032784FB3F
:100D340093074000631AF700832704FC0327C4FBCE
:100D440023A0E7006F00401AEFF05FD96F00C019CD
:100D5400034744E9930720076318F718232E04FC7C
:100D6400930744E993872700130744F99305070081
:100D740013850700EFF01FA02324A4FC832744F964
:100D8400130744F99305070013850700EFF09F9EAE
:100D94002322A4FC032744FC930710006310F702EA
:100DA400832784FC83C70700232EF4FCB7170000B5
:100DB40013858737EFF08FC56F008005032744FC48
:100DC400930720006310F702832784FC83970700AE
:100DD400232EF4FCB717000013850738EFF00FC378
:100DE4006F000003032744FC930740006310F702DD
:100DF400832784FC83A70700232EF4FCB717000085
:100E040013858738EFF08FC06F008000EFF01FCD9F
:100E1400032744FC93071000630EF700032744FCE8
:100E2400930720006308F700032744FC930740005E
:100E3400631CF70A832784FC1389070093D7F741BF
:100E440093890700930744E913070003930680007E
:100E5400930509001386090013850700EFF04FE797
:100E6400930744E913850700EFF04FBAB717000062
:100E740013850739EFF08FB9930744E98325C4FD3F
:100E840013850700EFF08FCC930744E9138507001F
:100E9400EFF0CFB7B717000013854739EFF00FB75E
:100EA4008327C4FD138A070093D7F741938A070069
:100EB400832744FC93961700930744E91307000320
:100EC40093050A0013860A0013850700EFF04FE02C
:100ED400930744E913850700EFF04FB3B7170000F9
:100EE40013858739EFF08FB213000000EFF00FA0E5
:100EF40093070500E38C07FE6FF09FC9972100005C
:100F0400938101CB138541C3138681C53306A64063
:100F140093050000EF0080040325010093054100C0
:100F240013060000EFF09FC16F004000130101FFA2
:100F340093050000232481002326110013040500D7
:100F4400EF00800F03A581C28327C50363840700D4
:100F5400E780070013050400EF0080301303F0005E
:100F640013070500637EC3029377F7006390070AB3
:100F740063920508937606FF1376F600B386E600BF
:100F84002320B7002322B7002324B7002326B70069
:100F940013070701E366D7FE6314060067800000A9
:100FA400B306C3409396260097020000B38656000A
:100FB4006780C6002307B700A306B7002306B7005F
:100FC400A305B7002305B700A304B7002304B700A3
:100FD400A303B7002303B700A302B7002302B7009B
:100FE400A301B7002301B700A300B7002300B70093
:100FF4006780000093F5F50F93968500B3E5D5005F
:1010040093960501B3E5D5006FF0DFF693962700BC
:1010140097020000B386560093820000E78006FA28
:1010240093800200938707FF3307F7403306F600E7
:10103400E378C3F66FF0DFF3130101FD232C4101C4
:1010440003AA81C2232021032326110203298A141F
:101054002324810223229102232E3101232A5101C8
:1010640023286101232671012324810163000904DB
:10107400130B0500938B0500930A10009309F0FFEE
:10108400832449001384F4FF6342040293942400EC
:10109400B304990063840B0483A744106380770529
:1010A4001304F4FF9384C4FFE31634FF8320C102C6
:1010B4000324810283244102032901028329C101FB
:1010C400032A8101832A4101032B0101832BC100DF
:1010D400032C81001301010367800000832749006A
:1010E40083A644009387F7FF638E870423A204003A
:1010F400E38806FA8327891833978A00032C49006A
:10110400B377F70063920702E780060003274900DC
:1011140083278A1463148701E38427F9E38807F893
:10112400138907006FF0DFF58327C91883A54408E6
:101134003377F700631C070013050B00E7800600F4
:101144006FF0DFFC232289006FF09FFA13850500FE
:10115400E78006006FF09FFB130101FF2324810049
:10116400B7270000372400009387873A1304C43A52
:101174003304F44023229100232611009354244085
:10118400638004021304C4FF3304F40083270400BF
:101194009384F4FF1304C4FFE7800700E39804FE7C
:1011A4008320C10003248100832441001301010131
:1011B40067800000930505009306000013060000F5
:1011C400130500006F00400003A781C28327871422
:1011D400638C070403A747001308F001634EE80675
:1011E4001318270063060502338307012324C30869
:1011F40083A88718130610003316E600B3E8C80066
:1012040023A417192324D310930620006304D502C2
:101214001307170023A2E700B387070123A4B7002D
:1012240013050000678000009307C7142324F714F4
:101234006FF05FFA83A6C7181307170023A2E7000D
:10124400B3E6C60023A6D718B387070123A4B700C3
:1012540013050000678000001305F0FF678000009D
:101264009308D00573000000634405006F0000007C
:10127400130101FF23248100130405002326110018
:1012840033048040EF00C000232085006F0000007D
:0812940003A501C367800000FF
:10129C002020000020202000200000002D00000055
:1012AC0020207C007C0A00000A0D00002020642015
:1012BC003C616464723E202D2D20646973706C61F6
:1012CC0079206D656D6F7279200A000020206220F4
:1012DC003C62617564726174653E202D2D207365CE
:1012EC0074206261756472617465200A00000000EC
:1012FC00202072203C616464723E203C77696474E7
:10130C00683E202D2D2072656164206D656D6F72B5
:10131C007920776F72640A00202077203C61646426
:10132C00723E203C76616C75653E203C7769647436
:10133C00683E202D2D207772697465206D656D6F68
:10134C00727920776F72640A000000002020202040
:10135C0077696474683D312C2032206F7220340A16
:10136C00000000003E3E00000A0D3A006368617206
:10137C002040000073686F7274204000696E742006
:10138C0040000000203D200028000000290A0D002C
:04239C00000000003D
:0823A00074000000D0000000F1
:0423A8008C000000A5
:1023B000000000009C260000042700006C2700009D
:1023C000000000000000000000000000000000000D
:1023D00000000000000000000000000000000000FD
:1023E00000000000000000000000000000000000ED
:1023F00000000000000000000000000000000000DD
:1024000000000000000000000000000000000000CC
:1024100000000000000000000000000000000000BC
:1024200000000000000000000000000000000000AC
:10243000000000000000000000000000000000009C
:10244000000000000000000000000000000000008C
:10245000000000000000000001000000000000007B
:102460000E33CDAB34126DE6ECDE05000B00000040
:10247000000000000000000000000000000000005C
:10248000000000000000000000000000000000004C
:10249000000000000000000000000000000000003C
:1024A000000000000000000000000000000000002C
:0C27D800B0230000000100F0B02300005E
:0400000300000F00EA
:00000001FF
